:020000040000FA
:10000000000C0400000000000418000004180000A8
:100010000418000004180000041800000418000070
:100020000418000004180000041800000418000060
:100030000418000004180000041800000418000050
:100040000418000004180000041800000418000040
:100050000418000004180000041800000418000030
:100060000418000004180000041800000418000020
:100070000418000004180000041800000418000010
:100080000418000004180000041800000418000000
:1000900004180000041800000418000004180000F0
:1000A00004180000041800000418000004180000E0
:1000B00004180000041800000418000004180000D0
:1000C00004180000041800000418000004180000C0
:1000D00004180000041800000418000004180000B0
:1000E00004180000041800000418000004180000A0
:1000F0000418000004180000041800000418000090
:10010000041800000418000004180000041800007F
:10011000041800000418000004180000041800006F
:10012000041800000418000004180000041800005F
:10013000041800000418000004180000041800004F
:10014000041800000418000004180000041800003F
:10015000041800000418000004180000041800002F
:10016000041800000418000004180000041800001F
:10017000041800000418000004180000041800000F
:1001800004180000041800000418000004180000FF
:1001900004180000041800000418000004180000EF
:1001A00004180000041800000418000004180000DF
:1001B00004180000041800000418000004180000CF
:1001C00004180000041800000418000004180000BF
:1001D00004180000041800000418000004180000AF
:1001E000041800000418000004180000041800009F
:1001F000041800000418000004180000041800008F
:10020000FFFFFF00FFFFFF000418000004180000BC
:10021000041800000418000004180000041800006E
:10022000041800000418000004180000041800005E
:10023000041800000418000004180000041800004E
:10024000041800000418000004180000041800003E
:101800000F802000007F22000001880000000000FF
:101810000C000700208021000100200011000700BB
:10182000000020000000E000020032000000020082
:1018300000000000C40C0200000000000040DA00BC
:101840000000FE004440A900407F20000000E000AE
:101850000300320000002000A00188004440A800DE
:101860000000060091018800800078000000EB0075
:1018700015003700E280400032A0B4009101BA00A8
:10188000E280400032A0B4009102BA00E280400041
:1018900032A0B4000002EB00472BDE00F507B200D7
:1018A000602CE10004003A000059EB008301E900DC
:1018B000FDFF3E00040037006128E1000100320016
:1018C0000082EB00040007001101BA000200E000F2
:1018D000E8FF3A00000006003159BA008301E90030
:1018E0000C0032002159BA008301E90008003200DF
:1018F0000400E00003003A00E280400032A0B4009F
:10190000F5FF370011D9BA008301E900FAFF3A0068
:101910008100E800E180400032A0B4000000060031
:101920000008BB00200424000C0007000000060093
:10193000821F780002042000B0C8BB00B058BB0072
:10194000B058BB000201E900FBFF3A001000240080
:10195000020007004F01780000000600003B8800ED
:1019600050052000303B8800A00A2000303B880052
:1019700061E7A800000000000000000061E7AF0080
:10198000FEFF370000000600C400FA00C100070097
:10199000C222A800AE00070090C5B3009100070066
:1019A0000004E0002700320050C4B3008D0007009F
:1019B0000004E0002300320030C5B30089000700B6
:1019C0000004E0001F003200E0602900EF00070083
:1019D000E0602900ED000700F0602900EB0007003F
:1019E000B0622900D300070000402A00160107005A
:1019F00040632900CF00070000802A00C8FF0700CD
:101A000080632900E1000700B0622900C9000700D7
:101A100000802A000C01070040632900C500070070
:101A200000802A00BEFF070080632900D70007005E
:101A3000E0632900BF0007000000EB0010079800DA
:101A400026003700B0642900D0000700E0602900BC
:101A5000CE000700CFFF37001E0090000043B0000B
:101A60001E01070000C2B3001C0107000000EB00CC
:101A7000000F78000B0037001E0178009E009000D8
:101A8000000C20000088B9009E004000E000290002
:101A900000804000904078006400470001717800A9
:101AA0001E0FE800F00B20009E0F1000F2FF340024
:101AB0001E0090004700DD008000780000802A00B2
:101AC00000804000800078006400470098FF070015
:101AD0001E0090000000E800100798001E00900013
:101AE000E70F5000DCFF340020662900A700070044
:101AF000706629008F0007000000EB0088FF0700D8
:101B000080632900A1000700906729008900070071
:101B10000000EB00000F7800050037001E01780080
:101B2000E400470000C0EB0000F178001E0FE80061
:101B3000F00B20009E0F1000F8FF3400E400470077
:101B400040C0B30080487800E40047000040EB004C
:101B500090409800E400470080CAB300A04098007D
:101B6000E40047000040EB00B0409800E40047006C
:101B70000040EB00C0409800E40047000040EB004C
:101B8000D0409800640047008000EB0068FF070029
:101B9000206629007D000700E06029007B00070027
:101BA000B068290079000700406929007700070024
:101BB000A06D290075000700C222A800A0CFB300C5
:101BC000D0000700A0CFB300CE000700C222A900BA
:101BD000A0CFB300CB000700A0CFB300C90007001F
:101BE000F5FF37000600FA002047980002010700C1
:101BF000004F78001E407800B800070000C6B30010
:101C00009E4F100007003600A0C7B3009E4F100083
:101C100004003E001E40780001CEB30001404000A9
:101C2000004F78002E4090009E4F500003003A0075
:101C30001000200020079800020037000000EB0091
:101C4000200798002E0090000080FA000000060097
:101C50000000FA00E06029004C00070070732900C2
:101C60004A00070030762900480007000077290065
:101C700046000700D079290044000700207C290095
:101C800042000700E0602900400007000080FA00E1
:101C9000000006000000FA004507A9000080EB00E4
:101CA000601988004227A900416A2000914078000D
:101CB00000CEB30000C060005040B300A4E6B700FF
:101CC000416C20009140780000CEB30000C060005D
:101CD0003040B300C4E6B700C922A800C902A8007A
:101CE000C8E2A800C8C2A800C942A800C222A90030
:101CF000C022A900CB62A900C962A900C002A90044
:101D0000C202A90020022000401188000000EB0060
:101D1000001188002062A8000000EB00101188006C
:101D200021E2A8002342A8008560A9000080FA00F3
:101D3000000006000600FA001007980002003700B5
:101D40001E407800650007001E009000104F7800CC
:101D50001E407800404798004E4090000004E0008C
:101D60000200320010C0B300404798004E4090007F
:101D70009E0090008100E800110798000004E00038
:101D8000EFFF3A000080FA00000006000600FA00AB
:101D900010079800020037001E4078004F0007002F
:101DA0001E009000104F78001E40780040479800B9
:101DB0004E4090000004E0000200320010C0B3006A
:101DC000404798004E4090009E0090008100E8003F
:101DD000110798000004E000EFFF3A00D0C0B30004
:101DE0003E000700A0C0B3003C0007000080FA00DE
:101DF000000006000400FA0010079800F07F290098
:101E0000CCFF07001E0090004400DE006F0F600052
:101E10009E007800F07E290000804000104078008D
:101E20002E0007001E0090006F0F60009E007800DB
:101E3000F07E290000804000104078002700070055
:101E40000080FA00000006000400FA001007980065
:101E5000F07F2900B7FF07001E0090004C00DE0055
:101E60006F0F60009E007800F07E29000080400027
:101E700010407800190007001E0090004800DE00A6
:101E80006F0F60009E007800F07E29000080400007
:101E900010407800110007001E0090004400DE0092
:101EA0006F0F60009E007800F07E290000804000E7
:101EB00010407800090007001E0090006F0F6000BE
:101EC0009E007800F07E29000080400010407800DD
:101ED000020007000080FA00000006000200FA007D
:101EE000004F780023C2BF00624060000004E000A1
:101EF000FCFF3A001E00FB00201188000080FA0061
:101F0000000006000600FA00404798000040EB0081
:101F1000204798000E0037000000EB00000F78000B
:101F200005003700A0CFB3000F0007001E007800A7
:101F30000000E800000F78001E007800E30F50005A
:101F4000F8FF36002E4090000040E800204798003F
:101F5000AE4090004E40900080CF5000EEFF390020
:101F60000080FA00000006000400FA0020479800F4
:101F70000040EB00004F7800130037000000000025
:101F80000000000000000000000000000000000051
:101F90000000000000000000000000000000000041
:101FA0000000000000000000000000000000000031
:101FB0000000000000000000000000001E4078004B
:101FC0000040E800004F78009E4078002E409000CE
:101FD00080CF5000E9FF39000080FA0000000600C1
:101FE0000000FA0022C2BF00614060000080FB00D8
:101FF0000080FA00000006000000FA0022C2BF00C4
:10200000614060000004E000FCFF320030118000FD
:102010000080FB000080FA0000000600202F000076
:102020008CA9000042270000A945000007AE00006F
:1020300042A7000037FE0000FF2F0000F0FF000065
:102040008860000019A90000CC220000A8C8000088
:1020500022A8000068A00000A9CC000002A900008E
:10206000C8020000000000000000000000000000A6
:10207000AFCA000022370000860000008026000062
:102080003580000027360000A8A4000006A9000043
:10209000A4260000A8A4000046A90000A466000031
:1020A000A9A4000086A80000C4060000A8C400007F
:1020B00026A90000C4460000A9C4000066A90000CB
:1020C000C4860000A8C4000022A90000C0220000AD
:1020D000EB8000000020000010020000884000009B
:1020E00011A8000020620000A8210000E2A8000062
:1020F00023420000075B000000B10000100C00004C
:102100003A66000000200000400D0000882000001A
:1021100011200000100000008820000011200000A5
:10212000200000008820000011200000B004000002
:102130008820000011EB000000070000074F00009E
:102140000088000090010000074D000000B700006B
:1021500003E10000074B000000B7000002E10000AF
:10216000BF020000817800008002000078000000BB
:10217000020700004600000078800000060700000B
:102180004400000078800000012000000280000070
:10219000074100000078000000590000E9830000BA
:1021A000013A0000FCFF0000E00E000004320000D5
:1021B0000300000020E0000004880000201100005F
:1021C00037E80000FF200000028000002A03000022
:1021D00080E100000328000031030000002A000015
:1021E000037C0000E103000028360000040000002A
:1021F000EB800000002000000005000088200000A7
:1022000011370000DDFF0000A70D000010370000AF
:10221000020000002FF10000FF370000D7FF000090
:10222000A60100000037000004000000BB8500008C
:102230000A24000020040000071A000000EB000040
:10224000800000002003000004BB0000B2CA0000B0
:10225000BBB200005ABB0000B25A0000E983000084
:10226000013A0000FBFF00002410000000070000FE
:102270001100000020030000042000000280000084
:10228000BA140000C0E10000320400003A09000066
:1022900000BA000034400000E1320000043A0000BF
:1022A00006000000BA34000040E1000032040000E3
:1022B0003A03000000E90000830100003AF5000045
:1022C000FF370000BBFF0000206000000588000011
:1022D0002011000037BA0000FF880000003B00001A
:1022E0002050000005880000303B000020A00000C6
:1022F0000A880000303B0000A8610000E7000000F1
:10230000000000000000000000AF000061E70000D6
:1023100037FE0000FF06000000000000200A000059
:1023200000EB000080050000FE00000060AE000031
:10233000220200003703000000800000301100007E
:10234000470000000706000000000000E98B0000C5
:10235000053A0000F8FF0000E90A0000053A000015
:10236000F5FF0000202F00008CA900008560000010
:10237000A985000080A9000023420000A9210000D7
:10238000E2EF000002210000A9C4000022A8000022
:10239000C022000088260000358800002736000093
:1023A000A9680000A0A80000C802000020000000EA
:1023B000008800006019000037630000FF00000083
:1023C0000008000000C20000000000000000000043
:1023D0000000000000FE000000000000FFFF000001
:1023E000FFFF0000FFFF0000FFFF0000FFFF0000F5
:1023F000FFFF0000FFFF0000FFFF0000FFFF0000E5
:10240000FFFF0000FFFF0000FFFF0000FFFF0000D4
:10241000FFFF0000FFFF0000FFFF0000FFFF0000C4
:102C100000DF0000F90000007F3F000000530000CB
:102C20006974000020620000616300006B200000F6
:102C3000616E000064200000656E00006A6F000095
:102C400079200000746800006520000073680000AF
:102C50006F7700000045000072610000736900009A
:102C60006E670000200000002E2E00002E000000E5
:102C7000206400006F6E00006500000057720000C5
:102C800069740000696E000067200000726F000028
:102C900077200000002000002020000020550000C8
:102CA000706700007261000064650000206300002E
:102CB000616E0000636500006C6C000065640000DC
:102CC0002E000000646F00006E65000000450000EB
:102CD00072610000736900006E6700002030000020
:102CE0007830000030300000302E00002E2E000022
:102CF0000057000072690000746900006E670000F0
:102D0000207200006F770000203000002E2E00009F
:102D10002E20000000530000756300006365000072
:102D20007373000021000000557000006C6F0000FC
:102D30006164000020760000342B00002066000053
:102D4000697200006D77000061720000652000006C
:102D50007769000074680000207400006865000056
:102D60002064000073330000302000004C6F00002E
:102D70006164000065720000206100007070000056
:102D8000207400006F200000636F00006D70000071
:102D90006C65000074650000207400006865000028
:102DA000207500007067000072610000646500001B
:102DB0002E0000004C6900006768000074200000CD
:102DC000757000002061000020630000616E00004B
:102DD000646C0000652C0000207300006179000025
:102DE000206C00006F740000732000006F6600000C
:102DF00020700000726100007965000072730000AD
:102E00002C2000006B650000657000002079000038
:102E10006F75000072200000666900006E67000098
:102E20006572000073200000637200006F73000081
:102E300073650000642C0000206100006E640000D7
:102E400020720000657300006574000020790000A6
:102E50006F75000072200000627500007370000042
:102E60006972000061740000652E000000440000DB
:102E70005333000030200000426F00006F740000E8
:102E80006C6F000061640000657200002069000042
:102E90006E730000746100006C6C000065720000CD
:102EA00020760000302E000032200000287600003E
:102EB0006572000079200000414C0000504800007D
:102EC000412900000028000043290000687200002A
:102ED0006973000020320000303100003000000033
:102EE000526500006C6500006173000065640000BD
:102EF000207500006E640000657200002043000031
:102F000072650000617400006976000065200000B1
:102F1000436F00006D6D00006F6E000073200000B5
:102F20006E7500006C6C0000206C0000696300008E
:102F3000656E0000736500000054000079700000A9
:102F4000652000002759000065730000272000005D
:102F5000746F000020700000726F00006772000044
:102F6000616D00002074000068650000206E0000A4
:102F700065770000206C00006F6100006465000050
:102F8000720000006F72000020640000697300008E
:102F9000636F00006E6E0000656300007420000027
:102FA000706F000077650000722000006966000005
:102FB000207500006E73000075720000652000002F
:102FC000286E00006F20000068610000726D000034
:102FD000206400006F6E00006529000000300000D2
:102FE000313200003334000035360000373800003D
:102FF00039410000424300004445000046300000D3
:1030000078000000000000000000FE00FFFFFF004D
:10301000FFFFFF00FFFFFF00FFFFFF00FFFFFF00BC
:10302000FFFFFF00FFFFFF00FFFFFF00FFFFFF00AC
:10303000FFFFFF00FFFFFF00FFFFFF00FFFFFF009C
:10304000FFFFFF00FFFFFF00FFFFFF00FFFFFF008C
:020000040001F9
:0857F800DFF900007F3F000013
:00000001FF
